:10000000F0288030A100FE30A4200130A4207530FB
:10001000A6003030BB28A101A117AE00FE30A420FD
:100020002E08A428A401A900AA01A01124080319DC
:10003000A0151030A3000301A90DAA0D031801306B
:1000400045202308031D1B280800A401A900AA01BC
:10005000A01124080319A0150530A3002730A8001B
:1000600010303E200330A800E8303E20A801643064
:100070003E20A8010A303E2029084528A7002A086A
:10008000A6002908A500CF202508A500A303031971
:10009000A011240803194F28230203185628250805
:1000A000031DA011A0195628303EA4280800AC005A
:1000B000061186118316061186110F3086058312EC
:1000C0002C08A01881283E30A6008030BB20333099
:1000D000AB0095201330A6008830BB2095206430FB
:1000E000BA2095206430BA202230AB009520283009
:1000F00080200C30802006308020A0142C0881281D
:100100002014AB00201C8F288611033C031C94286C
:1001100094200530A600DC30BB2003140800201416
:10012000FE3C0319A2288615201C201006150F304E
:1001300086052B08F03986040611AB0E2018952889
:100140003230BA202C08EB28A11B572883178001D6
:10015000840AFF3E031DA728EB28A801A700FF3053
:10016000A707031CA807031CEB280330A600DF30F9
:10017000BB20AF28A601E83EA500A609FC30031C61
:10018000C428A5070318C128A5070000A60FC12889
:100190002518CA28A51CCE280000CE280800AA01D0
:1001A000A9011030AB00260DA90DAA0D2708A90240
:1001B0002808031C280FAA020318E5282708A90706
:1001C00028080318280FAA070310A50DA60DAB0BCE
:1001D000D3282508EB28831383120313000008009B
:1001E000A00107309F00F03083168500FF308600A5
:1001F00081132030840060308312A720A030840057
:100200005030A720203084003030A6200130A800D4
:10021000F430AE2001204430572065305720633041
:1002200057206F3057206430572065305720723088
:100230005720203057205720553057204B3057201B
:1002400020305720563057202D305720313057203E
:100250008030A100C0300B20773057205720572026
:100260002E30572070305720693057206330572088
:100270006230572061305720733057206930572043
:10028000633057202E3057206E3057206C30572067
:100290007A29B501051A3016051E30120301051A18
:1002A000013E301A013C03190130031D0301AF0068
:1002B000323035020130031803012F05031962297A
:1002C000B50A4E2932303502031D6729AC2AB01C0D
:1002D00075298310301E831483183016831C301246
:1002E0000230A6007130BB2079290430A6004C30C2
:1002F000BB200800051105108510B501051E8129D8
:100300007E290130051A0301AF0034303502013077
:10031000031803012F0503198F29B50A81293430E9
:10032000350203189429A62A3108B2003308B40014
:100330000515B501B101B301FF30350201300318D5
:100340000301AF000130051A03012F050319AA2983
:10035000B50A9C293010B01019303502031CBB2996
:100360005B3035020318BB29301431170530A60065
:100370000301BB20C5295B303502031CC129B01421
:10038000C5290830A6008430BB20B01CFB29051EFF
:10039000CA29C729051ACD29CA29051ED029CD2960
:1003A000051AD329D029051ED629D3290730A6003E
:1003B000D030BB20051A8515051E8511051AB0150C
:1003C000051EB0110301B019013E051A013C031DC1
:1003D000EA29E2290430A6004C30BB204921B3179A
:1003E000301EB31349213317301E33134921B3167E
:1003F000301EB312FF2949218515301E8511492170
:100400003316301E33124921B315301EB311492162
:100410003315301E33114921B314301EB310492156
:100420003314301E3310B01C1D2A4921B117301E61
:10043000B11349213117301E31134921B116301E35
:10044000B11249213116301E31124921B115301E29
:10045000B11149213115301E31114921B114301E1D
:10046000B11049213114301E311033083402031DFC
:100470000130AF0031083202031D01302F04AF00FC
:100480000301B018013E3019013C031D01302F0457
:100490000319A22A0120301C562A5230572043301B
:1004A00057203530572058305720652AB01C5F2A16
:1004B000523057204330572036305720652A52306B
:1004C00057204330572035305720203057205030A8
:1004D0005720723057206F305720743057206F30BC
:1004E0005720633057206F3057206C30572003302F
:1004F000A800E830AE200120533057207930572033
:10050000733057203A3057208030A100330825201F
:100510008030A10088300B20330812208030A100E9
:10052000C0300B20433057206F3057206D3057209C
:100530003A305720310825208030A100C8300B20E8
:10054000310812203015B01C30117A290514013001
:10055000A800F430AE207A29051185140130A800D6
:0E056000F430AE203208B1003408B3007A291E
:02400E00303F41
:00000001FF
